:020000020000FC
:100000000C94EC0ED0C100000000000000000000C5
:1000100000000000000000000000000000000000E0
:10002000000000002EC000000000000098C000008A
:1000300000000000000000000000000000000000C0
:10004000A1C000000000000000000000000000004F
:100050000000000002030406080C10182030406065
:1000600080000406080C10182030406080A0C000FA
:100070000003070F1F000D0D04050D050205030306
:1000800002004FB662FD0DC0552049F00994C52D00
:10009000C095089483FDC795C093B20064604FBEBD
:1000A0001895C0910401089483FDC795C093B200D0
:1000B0006B7FC0910401CF3F09F419C04FBE2B984C
:1000C0002C982D9818952B982C982D9876FD0DC06E
:1000D00065FD0BC0C5E0CA95F1F7C0915101C0FDA7
:1000E0002A9AC1FD289AC2FD299A4FBE18952092DE
:1000F000B200CC27C160C7BB6460F7CFC8CF70FF28
:10010000C6CF65FDC4CF2B9AC2CF70FFC0CF65FDAF
:10011000BECF2C9ABCCF70FFBACF65FDB8CF2D9A59
:10012000B6CF2A9870FFB3CF65FDB1CFC1E4CA95B1
:10013000F1F72B9AACCF289870FFA9CF65FDA7CF18
:10014000C1E4CA95F1F72C9AA2CF299870FF9FCFEE
:1001500065FD9DCFC1E4CA95F1F72D9A98CF4FB6B2
:10016000C0916F00CD7FC0936F006E7FC0918400FF
:10017000CE0DD0918500DF1DD0938900C0938800FB
:100180004FBE18953FB68F7EADB3A170A2118061AE
:10019000A0E0ADBBA0916E00AE7FA0936E007894FE
:1001A000A0910801AA2341F085FD2BC0A091080170
:1001B000AA95A093080125C040E050E085FD15C038
:1001C000A9B196FDA095A2FD4FEFA3E096FDA2E098
:1001D000A0936900AA27A160ACBB8D7FA9B196FD51
:1001E000A095A2FD5FEF451739F7A8E161FDA09347
:1001F000080185FD03C0A8E1A093080140933601E2
:10020000816085FD0EC0A0910901AA2331F0A09163
:100210000901AA95A093090104C08061AA27A160E1
:10022000ACBB80FF3CC0A09136014A2F61FF8E7F9E
:1002300085FD1CC0A0915401A430C1F4403F08F0DA
:1002400040EFA42FA295AF704A0F50915601533042
:1002500069F0A695A69550FD01C0A69552FD03C074
:10026000A41B4A2F03C04A0F08F44FEF409301012B
:10027000A72FA670A1F073FD12C0A0911001AA0FC4
:10028000AA0F50913E0156955695541708F0452FE8
:100290004A0F4093010118F4AFEFA0930101409180
:1002A0005401443009F03AC0A0910101A093030128
:1002B00040910301A0913B014A1708F04A2FA091F9
:1002C0003D014A1708F04A2F542EA0914001AA235D
:1002D00009F422C0542F5A1B10F4A42F50E0BA2E58
:1002E0008894AA1FAA2EA0914201A095AA22A50E29
:1002F00058F0A0914101A21509F0AA95AA0EA09369
:10030000410148F04A2D08C0A0914101BA1608F0F9
:10031000A395A09341014FEF40930401A52DA03474
:1003200008F06860A0910001A395A093000161F01E
:10033000F894A0916E00A160A0936E0084FF02C0AB
:10034000A1E0ADBB3FBE1895A0911401A395A09369
:10035000140141E050910801552329F085FF03C0A5
:100360005A9550930801A0913601A13018F02092BF
:1003700039010DC020923A0120924301A091390128
:10038000AF5FA093390118F0AFEFA0933901F89453
:10039000A0916E00A160A0936E0084FF02C0A1E056
:1003A000ADBB3FBE18953FB640918400509185008B
:1003B0008F7EADB3A170A2118061A0E0ADBBA09112
:1003C0006E00AE7FA0936E00789481FD25C0A2E000
:1003D00096FDA3E0A09369008260A9B196FDA09567
:1003E000A2FF05C0409305015093060141C1A3E05F
:1003F00096FDA2E0A0936900AA27A160ACBB8D7F07
:1004000085FF01C028C140E0A9B196FDA095A2FDDD
:1004100022C14093360111C1A3E096FDA2E0A09352
:1004200069008D7F61FF72C0A2E096FDA3E0A093FA
:100430006900AA27A160ACBB826040933101509350
:100440003201A0902F014A19B09030015B09BB2402
:10045000A22C4C38520518F42092350149C0A091C5
:100460007401AA2359F1483C520528F4A0E1BA2EA0
:10047000AAE0AA2E23C04836A1E05A0728F4A8E033
:10048000BA2EAFE0AA2E1AC0403DA2E05A0728F4C7
:10049000A4E0BA2EAEE1AA2E11C0403AA5E05A0758
:1004A00028F4A2E0BA2EACE3AA2E08C04839A8E08E
:1004B0005A0720F4A1E0BA2EA8E7AA2EC42EA091D4
:1004C0003301CA1AD52EA0913401DA0ADD202AF4AC
:1004D000AFEFC094D094CA1ADA0A20923501A8E08E
:1004E000A210A0E0CA14DA0618F4A1E0A093350126
:1004F00040933301509334014091310150913201C6
:1005000040932F015093300142E097C0A091050124
:100510004A1BA09106015A0B94FD82C093FD80C036
:1005200092FD7CC086FF03C0D52EC42E0CC056950C
:10053000479591FD73C05695479590FD6FC0D52E98
:10054000C42ED694C79461FD19C0AC2DAC51AD2D0D
:10055000A24008F005C0DD2089F4AC2DA85C70F441
:10056000A0910701A395AA2311F0A0930701AA3037
:1005700008F471C02092360181606DC0A09107011E
:10058000AA2319F0AA95A0930701A22C50915A0111
:1005900097FD06C0A0906801533011F4A09070013F
:1005A000AAEFAA0EA22DA21DCA18DA0A4FB74170EF
:1005B000533049F4442321F087FD05C0806803C00F
:1005C00087FF01C08F77442359F0533031F4AFEFE8
:1005D000C094D094CA1ADA0A03C040E050E020C0A8
:1005E000533049F4CC0CDD1CAAE0CA1AD20818F426
:1005F000A0E0CA2ED22CAFEFCA16D20418F04FEFEB
:1006000050E00EC0A0914C01CA9E412D000C441F29
:1006100050E008F012C04FEF50E00FC056954795DC
:1006200094FF07C0552309F04FEFA42FA6954A0F5A
:10063000521D4F3F520508F04FEF40933601816045
:1006400061FF09C0AFE1A095A923AB299A2F8F7D47
:10065000BB2009F48062A8E1A093080185FF03C0D4
:10066000AAE0A093080161FD03C085FD01C08F7E53
:1006700085FD03C0A6E0A0930901F894A0916E0047
:10068000A160A0936E0084FF02C0A1E0ADBB3FBE9D
:10069000189511E00AC013E008C01AE006C01EE178
:1006A00004C014E602C018EC00C005E1BB27BA95EF
:1006B000F1F70A95D9F71A95C1F708952AE338E7B3
:1006C00009C020E33CE806C02AE234EB03C025E27F
:1006D00038EC00C012E0BB272898BA95F1F72C9AA5
:1006E000BA95F1F72C98BA95F1F7289ABA95F1F7DF
:1006F000123009F02B9A123009F42D9AB0914D0165
:10070000BA95F1F7123009F02B98123009F42D98B0
:10071000B7E8BA95F1F71A95F1F6022FB22FBA950C
:10072000F1F70A95D9F73A95A9F628980895221B6A
:1007300039E0001F3A9509F40895221F211B18F48F
:10074000210F8894F6CF0894F4CF622C722CB0E07D
:100750008894B395221F331FE0F737952795889427
:10076000912E802E020B130B10F4192D082D10F46E
:10077000889401C00894661C771CBA9571F7172DF0
:10078000062D0895322D11232AF43A9500951095DF
:10079000031B130BF894029F712C002D129F912CB8
:1007A000802C7894780C172D921C292DB4E06B2E98
:1007B0002695179507956A94D9F7332321F000956C
:1007C0001095031B130B0895009154010430A9F1F7
:1007D000B0913601B15008F010C0B0910101B09352
:1007E000030120921E0120921F01209220012092DD
:1007F0002101209222016F7B20C06090540160642F
:10080000B0910101B093020108E317EC20911A01A5
:1008100030911B0136952795B62DBA9541F0369546
:100820002795B62DBA95BA9511F0369527950E9461
:10083000A50300931E0110931F01089500911E014E
:10084000B09102010B1B10911F01120928F400380E
:10085000BFEF1B0740F009C00F37120508F405C0B1
:100860000FE710E002C000E81FEF00932301109390
:100870002401089500912301B09120010B0F1091E4
:100880002401B09121011B1F20E03091240133236A
:100890000AF42A95B09122012B1F1AF4203F40F050
:1008A0000AC02F3008F407C00FEF1FEF2FE003C07E
:1008B00000E010E020EF30910301B0913B013B17C5
:1008C00018F4323030F009C0B0912401BB235AF043
:1008D00004C0B0912401BB2332F400932001109393
:1008E0002101209322010895209177010091230195
:1008F000000F10912401111F0E94C20311232AF43A
:100900000038BFEF1B0740F009C00F37120508F48D
:1009100005C00FE710E002C000E81FEF002352F00F
:10092000B0910201B01B0B2F18F0013008F00AC083
:1009300001E008C000950F5FB09102010B0F08F0B5
:1009400001C00FEF009325010895209178010091D7
:100950002101109122010E94C20311232AF40130C7
:10096000BFEF1B0740F009C00F3F120508F405C098
:100970000FEF10E002C001E01FEF112352F0B09121
:100980002501B01B0B2F18F0013008F00AC001E060
:1009900008C000950F5FB09125010B0F08F001C052
:1009A0000FEF0093030108950FEF677F71FD2AC0D9
:1009B00072FD09C06860B0911B01BA3020F0B52DFE
:1009C000B03408F4677FB0917301BB23D9F0B091C4
:1009D0001B01BB23B9F00FEF10911B010E9497037D
:1009E000F894B091130172FDB5E00B9F112D002D0D
:1009F0007894112309F00FEFB0913E010B1710F41A
:100A000000913E0100933D01089500911A0110915B
:100A10001B0100541140B0913D0110F4BA9501C082
:100A2000B39511F0B0933D01089500C00895209151
:100A30005501B0917A00B6FDFACF0091780010917F
:100A40007900B0917A00BF77B0937A00B0914A01F3
:100A5000B395B0934A01B83060F120924A01B09149
:100A60007201BB2321F1112329F0B0914B01BF3F4B
:100A700061F009C0B0914B010B1739F020F4BB2392
:100A800021F0BA9502C0B395E1F300913B01B09318
:100A90004B01B03050F400ECB03038F400E8B03026
:100AA00020F400E4B03008F400E000933B017F7EC6
:100AB000089510913B01B0E11B0F08F41FEF109354
:100AC0003B01B0915401B43081F000913B01B091F1
:100AD0000301B01B10F400910301B0913D010B170D
:100AE00008F00B2F502E00930401B0914A01B7304B
:100AF00009F47061089502E3F894B09179010B9FB5
:100B0000012D000C001F7894B0913B010B1710F0E1
:100B100000913B010093010100930301502E0093CB
:100B2000040100933E01089520921A01B0EFB093A2
:100B30001B010895F8940091840010918500209184
:100B400014017894309115016090160100931501FD
:100B500010931601031B160971FD03C077FD7DC0BC
:100B600027C070901701209317012709222311F045
:100B70000FEF1FEF8090180190901901309318012A
:100B800060921901009115011091160108191909B7
:100B900020911A0130911B0136952795020F131FE2
:100BA00010F40FEF1FEF00931A0110931B0129C0DF
:100BB00020911A0130911B013901B4E08B2EB2E073
:100BC0009B2E343010F08A949A94383010F08A9426
:100BD0009A94769467948A94E1F7261937099920B4
:100BE00021F0169507959A94E1F7200F311F209375
:100BF0001A0130931B0128F43FEF30931A01309310
:100C00001B01323008F4706871FF02C0B3E00DC000
:100C1000B091640100911101023838F0B395003AA7
:100C200008F0B395B63008F0B5E09B2EB4E08B2EFB
:100C300010911B0100911A0124E0169507952A9541
:100C4000E1F70819120928F0B02FB250B12FB209FC
:100C500010F402E010E0980126C020911A013091B2
:100C60001B013901769467946694669466942619FC
:100C7000320906950695200F321D20931A013093F4
:100C80001B01323008F07F7704E0369527953695C2
:100C9000279526952695201B10F0223008F422E097
:100CA00089019090640160FDFECFE0902B01F090EF
:100CB0002C016160B0916F00B260B0936F00380199
:100CC00077FD41C07694679400932B0110932C011B
:100CD000B92DB330E1F0B0FD04C0060D171D93012E
:100CE00006C0000F111F0250120922E030E0B92D9A
:100CF000B33068F020932D0130932E01009327012B
:100D0000109328016092290170922A013AC0009341
:100D10002D0110932E01209327013093280160921A
:100D2000290170922A0171FF0DC0BFE0B0932D011F
:100D300020922E01B093290120922A01B0932B0119
:100D400020922C011EC0669400932B01B92DB33064
:100D500091F0B0FD03C0060D262D03C0000F025018
:100D600022E0B92DB33038F020932D0100932701F4
:100D70006092290106C000932D0120932701609203
:100D8000290100911C0102FD0350013039F495FD49
:100D90000EC0B5E0B06CB0937C000DC0023029F4F9
:100DA000B4E0B06CB0937C0006C095FDF2CFB3E028
:100DB000B06CB0937C0000914201000F10F4BBE6D0
:100DC0000B270093420160FDFECFB2E0B0930E010D
:100DD0006160B0916F00B260B0936F00B72FB670D2
:100DE00001F120911A0130911B0136952795369516
:100DF000279571FF02C0B0E43B0FF8940091840086
:100E000010918500020F131F109389000093880032
:100E10006160B2E0B6BBB0916F00B260B0936F009A
:100E200078940895606120921D0120E067FD20E222
:100E300006C0606120921D0120E267FD20E001E014
:100E400011E077FD11C0B72FB67009F06F7E14E185
:100E500000911B01069509F403950F3008F00FE08F
:100E600071FF02C004E114E160FD10C0B0911D01EA
:100E7000BB2361F071FF06C0B0910E01BA95B0932B
:100E80000E0111F4706252C00E94E806B0917B001E
:100E9000BF7BB0937B00B0B7B0917B00B064B093E0
:100EA0007B00B0911D01B395B0931D01B0B777FDE4
:100EB00006C0B1E071FDB3E0BA95F1F7B0B7B0721A
:100EC000B21709F028C071FF05C00395011708F09B
:100ED0000A95CACF64FD05C00395011708F0AFCF8E
:100EE000C3CF6F7EF894309184006090850070903D
:100EF0001A0180901B01370D681C609289003093A5
:100F000088006160B2E0B6BBB0916F00B260B09390
:100F10006F00789494CFB0910D01B13008F48FCF69
:100F200064FD8DCF0A9509F09FCF7F7D20912D0123
:100F300030912E01F894B2E0B6BB0091840010917C
:100F40008500020F131F1093890000938800E09022
:100F50002701F09028016160B0916F00B260B093FA
:100F60006F007894B72FB67039F0B0910D0172FF11
:100F7000B395B0930D0109C075FF07C067FD05C0AB
:100F800064FD03C0BF91BF918AC5089500E063FF6F
:100F900003C064FF01C001E0F89410911101B7E0B3
:100FA0001B9F212D102D7894200F2695179526959F
:100FB00017952695179510931101183718F4B8E76F
:100FC000B093110100911101B09112010B1720F0A3
:100FD00060622B982C982D9860FDFECFE09029013F
:100FE000F0902A016160B0916F00B260B0936F0021
:100FF0000895B2E095FD0AC0F894B0931C012898BA
:101000002A9A62FF01C02D9A7894F4C0F894B093A4
:101010001C012898299A62FF01C02B9A7894EAC093
:10102000B3E082FF24C095FD11C002E0F894B093B4
:101030001C01EBE9F0E0009351012D98299862FF23
:1010400002C02C9A01C0289A7894D4C002E0F89487
:10105000B0931C01EBE9F0E0009351012B982A9822
:1010600062FF02C02C9A01C0289A7894C3C095FDF3
:101070000BC0F894B0931C01E5E8F0E02D9862FFF6
:1010800001C02C9A7894B6C0F894B0931C01E5E89E
:10109000F0E02B9862FF01C02C9A7894ABC0B4E0CA
:1010A00095FD0AC0F894B0931C012A98299A62FF12
:1010B00001C02C9A78949EC0F894B0931C01299892
:1010C0002A9A62FF01C02C9A789494C0B5E082FFFE
:1010D00024C095FD11C001E0F894B0931C01E1E932
:1010E000F0E0009351012C98289862FF02C02B9ADF
:1010F00001C02A9A78947EC004E0F894B0931C0151
:10110000E5EAF0E0009351012C98289862FF02C0B4
:101110002D9A01C0299A78946DC095FD0BC0F89462
:10112000B0931C01EFE7F0E02C9862FF01C02B9A0E
:10113000789460C0F894B0931C01EBE8F0E02C9830
:1011400062FF01C02D9A789455C0B6E095FD0AC0A3
:10115000F894B0931C012998289A62FF01C02B9A39
:10116000789448C0F894B0931C012A98289A62FF9A
:1011700001C02D9A78943EC0B1E082FF24C095FD55
:1011800011C004E0F894B0931C01E5EAF0E000938C
:1011900051012B982A9862FF02C02D9A01C0299A0A
:1011A000789428C001E0F894B0931C01E1E9F0E0E4
:1011B000009351012D98299862FF02C02B9A01C01B
:1011C0002A9A789417C095FD0BC0F894B0931C012F
:1011D000EBE8F0E02B9862FF01C02D9A78940AC0EA
:1011E000F894B0931C01EFE7F0E02D9862FF01C086
:1011F0002B9A78946F7D08952EE730E0F9012092C4
:1012000051012B982C982D982A98289829986B7F13
:101210000895A2E5B1E009E00D9309E00D9304E023
:101220000D930FEF0D9303E00D930FEF0D930BE074
:101230000D9301E00D9301E00D9301E00D93AEE5F8
:10124000B1E001E00D930FEF0D930D930D930D930E
:101250000D9303E00D930FEF0D930FEF0D930D938F
:1012600005E20D9300ED0D9308E20D9300E50D935B
:1012700004E00D930FEF0D9302E00D9300E00D934A
:101280000AE70D930FEF0D9300E00D9301E00D932E
:1012900000E00D9303E00D9300E00D93089520917D
:1012A00059018B7FB0915A01B33019F09F7DB1FD88
:1012B00090629F7BB0915B01B1FD9064223011F090
:1012C000886001C0877F08950A95E00FF21DB491F0
:1012D0000895E4E5F0E0009152010E946409B093A2
:1012E0007701E4E5F0E0009153010E946409B093B6
:1012F0007801E2E6F0E0009158010E946409B093A1
:10130000790100915801023008F402E000931301C2
:10131000B0916E010FEFB23009F400EAB33009F476
:1013200002E800931201E0E7F0E0009175010E94ED
:101330006409B093400108950895209168013091A7
:101340006901B0915A01B33009F43E5097FF02C0D1
:1013500020E03FEFB32FB21B6B2EB25810F4B2E86F
:101360006B2E00E00395609EB12DBD57D8F300931E
:101370004C01089590680E949D090E944F0320E04F
:1013800030E0B0E16B2E0E944B03B09136012B0F81
:10139000321D6A94C1F7B4E036952795BA95E1F706
:1013A000822E9F770E949D090895F894E3E0F0E073
:1013B000B9E0B7BFB491B078C1F3F894A895B4B7C9
:1013C000B070B4BFB0916000B861B0936000B0E09D
:1013D000B0936000B4E0BEBFBFEFBDBF0E94FC0889
:1013E000B0E0B5B9BFE3B4B9B0E0B8B9B0E0B7B9EF
:1013F000B0E0BBB9B0E0BAB92224A0E0B0E02D92D1
:10140000AA31E9F7A0E0B1E00FEF2D920A95E9F7D4
:10141000B1E0B09342010E9409090E94920DB0E030
:10142000B06CB0937C00B0917A00B460B068B093B7
:101430007A0000916A0100934D01B1E0B0930A0176
:10144000F8940E9453030E945E030E944F030E947F
:1014500061030E944F030E9464030E944F03F894AB
:101460000AEF1AEFA9B196FDA095A2FF1FC01A9529
:10147000C9F70A95B1F7E0E0FCE3B591B43E39F461
:10148000B591B03E21F4B591BF3F09F40CC0E0E046
:10149000F395F395B591B83F49F4B591B43931F46A
:1014A000B591BA3A19F4EE27F69509940E944F09BE
:1014B0000E9469090E949C090E949D0900916A018D
:1014C00000934D010E94FC08B2E0B5BDB2E0B093BC
:1014D0008100B2E0B093B100B1E0B5BBB0936E0053
:1014E000B2E0B6BBB0936F00B1E0B7BBB093700091
:1014F000B0917B00BF7BB0937B00B0B7B0917B0015
:10150000B064B0937B000E94490378940E94150553
:1015100020921001B3E096FDB2E0B0936900B1E013
:10152000BDBBBB27B160BCBB8D7F0E945303626013
:1015300033E02CE0B0913501BB2321F42CE03A9547
:1015400009F48DCF0E944F0380FF89CF8E7FB09129
:101550003601B23070F3B92FBF710091380100939A
:101560003701B0933801B01721F72A9519F76D7F2D
:10157000B3E096FDB2E0B0936900BB27B160BCBB9D
:101580008D7FB0917401BB2321F48062B92FB070BC
:101590009B2F8F7B209207010E94510385FF05C07E
:1015A000B0910701BA3008F080640E944B0302E05A
:1015B00085FF01C000E0B0913601B017B0F3F89498
:1015C0000E945E030E945E030E945E0378940E9464
:1015D000530320922601B0915A01B33009F490C010
:1015E0000E944B03B0915E01B13008F489C0B09104
:1015F0000A01B13008F484C085FD1EC0B0913601E7
:10160000BF3F08F47DC0F8940E94670378940E945D
:101610005103B0913601B130B0F7F8940E945E03E7
:101620000E944D030E945E0378940E945103B09182
:101630003601BF3F90F368C3B3E09B2E9068F894E7
:101640000E949D0978940E945103F8949F770E940C
:101650009D0980903601B0913601BF37789408F427
:1016600057C00E944903F8940E94670378949A94A3
:1016700029F70E94BA09B82DB09369010E9453035B
:10168000F8940E94C50D0E94350E7894BAE09B2E06
:101690009068F8940E949D0978940E945103F894F0
:1016A0009F770E949D0980903601B0913601BF3727
:1016B000789460F70E944903F8940E945E030E94A8
:1016C0004D030E945E0378949A9411F70E94BA0920
:1016D000B82DBB5FB09368010E945303F8940E9439
:1016E000C50D0E94520E78940E945103F8940E94F6
:1016F0009D097894B0913601BF3F08F47DCF04C3B3
:1017000000913601B09126010B1710F000932601CD
:101710000E94510301E0B0915A01B35009F405E071
:10172000B0913601B01708F056CFF8940E946703C5
:101730000E9467030E94670378940E9453032092DB
:101740000A0120920B0120920C01B0910B01B3957C
:10175000B0930B01BF3F91F5B0910C01B395B093DD
:101760000C01B0916C0109E1BA9559F002E3BA9508
:1017700041F00DE7BA9529F00AEFBA9511F02092E1
:101780000C01B0910C01B017C8F00E94FC080E9437
:101790004903B0910C01BA95B0930C0120920B0152
:1017A000B0916B01B0934D01F8940E946703789457
:1017B000B0916A01B0934D010E9451030E944D0304
:1017C000B0910801BB2319F485FF01C048CE01E0A8
:1017D00085FD01C006E0B0913601B01708F4B5CF21
:1017E000B0915A01B35011F00E945103B091080119
:1017F000BB2309F434CEF8940E94FC082092010126
:101800002092020120920301522C20920401209286
:1018100041017894B0915701BB0FB0933F012092E2
:101820001E0120921F01209220012092210120926E
:10183000220120924A0160E070E020921101B8E09C
:10184000B0934A0170610E944903B0E074FDB0E0BA
:10185000B06CB0937C00B0917A00B068B064B09383
:101860007A00B0917A00B6FDFCCF0091780010911B
:101870007900B0917A00BF77B0937A00112309F014
:101880000FEF00934B010E941705B8E0B0934A0197
:1018900070610E944F09F894BFEFB0933B010E9422
:1018A0007B05B0910101B0933B01B0933C01B09333
:1018B0003D017894B1E0B0930101B09303015B2E38
:1018C000B0930401B0934401B0913A01B093430145
:1018D000B0915A01B33019F49F7D87FD9062716019
:1018E000726020920D010E94A5080E94BC080E940F
:1018F00094050E949A050E9494050E949A050E94F0
:1019000094050E9419070E94E4030E94C6070E94E2
:10191000F9070E949A050E94120766FD0E941E04A4
:1019200077FF0E94D40477FD0E9405050E94C60738
:101930000E9410080E949A050E94190766FD0E94E5
:101940003A040E94C6070E944F080E949A050E940E
:10195000120766FD0E9474040E94C6070E94660872
:101960000E949A050E94190766FD0E94A5040E9424
:10197000C6070E94A5080E949A050E941207B0E0BF
:1019800074FDB0E0B06CB0937C00B0917A00B068A8
:10199000B064B0937A000E94C6070E94BC080E94FF
:1019A0009A050E94170571FF24C0B0913E01B093C3
:1019B0003B01B0933C01B0913A01B0934301B1E0D7
:1019C000B093440118E12CE0B0910D01B11758F02B
:1019D0007D7F746020930F01B0913E01B0933B0175
:1019E000B0933D0106C0B0913601B13008F089CF07
:1019F00060C072FF11C067FD0FC0B0910F01BA95B2
:101A000019F47B7F78607DCFB0930F01B0913601E0
:101A1000B13008F076CF4DC020921001B09139015D
:101A20000AEF10917601112309F003E0B01708F0D6
:101A300040C085FF04C0B0910801BB23D1F1B09133
:101A40005A01B33081F495FD03C087FD04C00BC07B
:101A500087FF01C008C067FD06C06068B0913E0105
:101A6000B0933B0174CF00EF67FF05C0B0913E011A
:101A7000B0933B0100E2B0911B01B01708F441CFD5
:101A800067FF17C06F779F7D87FD90627460B2E13A
:101A9000B0930F01B0913E01B0933B0132CFB091B2
:101AA0001001B395B0931001B0913601BB2309F03A
:101AB00002C020921001F8940E94FC088090590105
:101AC000B2E0B09359010E944F09809259012092CF
:101AD00001012092020120920301522C2092040164
:101AE00020923F0160E070E078940E9451030E94D0
:101AF000FC0800917601002319F02B9A2C9A2D9A5C
:101B0000B0E0B06CB0937C00B0917A00B460B06883
:101B1000B0937A0085FF05C0B0911001B43008F091
:101B20009ECC0FCEEDE0F0E00E94BE0D053509F031
:101B30001EC0EEE0F0E00E94BE0D0A3A09F017C0A8
:101B40003AE0A2E5B1E0E3E0F0E00E94BE0D0D93C3
:101B500031963A95D1F739E1AEE5B1E0EFE0F0E04A
:101B60000E94BE0D0D9331963A95D1F704C00E94A4
:101B700009090E94C50DE8E2F0E00895F999FECF49
:101B8000E1BDF2BDF89A00B508950E94E80D3AE073
:101B9000A2E5B1E0E3E0F0E00D910E94E00D3196A6
:101BA0003A95D1F739E1AEE5B1E0EFE0F0E00D9123
:101BB0000E94E00D31963A95D1F70E94F30D0895F9
:101BC000F999FECF00BDE1BDF2BDFA9AF99A0895E8
:101BD000EDE0F0E00FEF0E94E00DEEE0F0E00FEF3F
:101BE0000E94E00D0895EDE0F0E005E50E94E00DB3
:101BF000EEE0F0E00AEA0E94E00D089530914E0117
:101C000000914F01313011F400935201323011F440
:101C100000935301333011F400935401343011F424
:101C200000935601353011F400935801363011F409
:101C300000936401373011F400935901383011F4E6
:101C400000937501393011F400936E013A3011F4AC
:101C500000935A013B3011F400935B01089525E095
:101C60000E9453032A95E1F708950E945E030E94A3
:101C700061030E9464030E9467030E944D030E9457
:101C80005E030E9461030E9464030E9467030E9436
:101C90004D030E945E030E9461030E9464030E9440
:101CA000670308950E9467030E9464030E94610312
:101CB0000E945E030E944D030E9467030E9464031A
:101CC0000E9461030E945E030E944D030E9467030D
:101CD0000E9464030E9461030E945E030895809045
:101CE0004E0190904F010E945E030E945E030E948D
:101CF0005E030E944D038A94B1F70E9467030E941D
:101D00004D039A94D1F70895F8940E94350E789473
:101D10000E942F0E0E942F0EB1E0B0934E01B1E051
:101D2000B0934F0120925001F8940E946F0E789466
:101D3000B5E06B2E709036010E945303B0913601CE
:101D40007B16C1F7B13018F0BF3F70F10CC00E9494
:101D5000FE0DF8940E94C50D0E94350EB8E0B093B8
:101D600060000E942F0E6A9429F7B0915001B3953C
:101D7000B0935001B33008F4D7CF0E942F0EB0912A
:101D80004F01B395B0934F01F894B0914E01BA95BD
:101D9000E6E7F0E0EB0FF21D049178940395B09123
:101DA0004F01B01708F4BECF0E942F0E0E942F0ED5
:101DB000B0914E01B395B0934E01B0914E01BC303D
:101DC00008F4ADCF0E940909F8940E94C50DB8E04F
:0A1DD000B09360000E942F0EE8CAD5
:00000001FF
